:100000000C94E6040C9403050C9403050C9403056E
:100010000C9403050C9403050C9403050C94030540
:100020000C9403050C9403050C941A260C94EC26EE
:100030000C9463200C9403050C9403050C940305A5
:100040000C9403050C9403050C9403050C94030510
:100050000C9403050C94EB200C9403050C940305FD
:100060000C9403050C9403050C9403050C940305F0
:100070000C9403050C9403050C9403050C940305E0
:100080000C9403050C9403050C9403050C940305D0
:100090000C9403050C9403050C9403050C940305C0
:1000A0000C9403050C9403050C940305BE08BE08CC
:1000B000EA08EA0852097009880A880A7B09140AC2
:1000C000250A250A59278027782880277828CC27D1
:1000D000EF2778284628552853005400550056002D
:1000E0005F006000610000005C005D005E00570082
:1000F00059005A005B0000000000620063005800D5
:1001000044454255473A2064697361626C65642EC8
:100110000A0044454255473A20656E61626C656449
:100120002E0A000A0025303258006C65645F746145
:10013000736B3A20004F6E6573686F743A20616389
:10014000746976653A2025640A000A002530386211
:10015000003A200025303258000A722F63203031D7
:100160003233343536370A00290A002575002F004E
:100170002575005D2800256400200025640020000E
:1001800025640020002564007C0025303258006D75
:100190006F7573656B6579205B62746E7C7820790E
:1001A000207620685D287265702F61636C293A2083
:1001B0005B00313A0964656C6179282A31306D73CE
:1001C000293A2025750A323A09696E74657276619A
:1001D0006C286D73293A2025750A333A096D6178C8
:1001E0005F73706565643A2025750A343A0974694D
:1001F0006D655F746F5F6D61783A2025750A353AD9
:1002000009776865656C5F6D61785F7370656564BB
:100210003A2025750A363A09776865656C5F746916
:100220006D655F746F5F6D61783A2025750A0070A7
:100230003A097072696E742076616C7565730A6430
:100240003A097365742064656661756C74730A7528
:10025000703A092B310A646E3A092D310A6C743AEE
:10026000092B31300A72743A092D31300A45534353
:100270002F713A09717569740A0A73706565642093
:100280003D2064656C7461202A206D61785F737015
:10029000656564202A2028726570656174202F20AE
:1002A00074696D655F746F5F6D6178290A77686541
:1002B00072652064656C74613A20637572736F7245
:1002C0003D25642C20776865656C3D25640A53657F
:1002D0006520687474703A2F2F656E2E77696B698C
:1002E00070656469612E6F72672F77696B692F4D36
:1002F0006F7573655F6B6579730A004D3E20004D25
:1003000025753A25733E20003F0A003D2025750AD9
:10031000003F0A0064656661756C74730A00257598
:100320000A003F0A000A092D2056616C756573208A
:100330002D0A00710A000A092D204D6F7573656B37
:100340006579202D0A003F00433E20004C25640AB9
:10035000000A092D20537461747573202D0A686F8B
:1003600073745F6B6579626F6172645F6C656473EF
:1003700028293A20253032580A6B6579626F6172FC
:10038000645F70726F746F636F6C3A2025303258FF
:100390000A6B6579626F6172645F69646C653A20AB
:1003A000253032580A74696D65725F726561643315
:1003B0003228293A202530386C580A000A092D20A5
:1003C00056657273696F6E202D0A5649443A203083
:1003D0007834423438284B6579486976652920504D
:1003E00049443A20307834443530286D6179706161
:1003F0006429205645523A203078303030310A4254
:1004000055494C443A202028466562203237203234
:10041000303232290A4F5054494F4E533A204C55EE
:100420004641204D4F5553454B4559204558545250
:10043000414B455920434F4E534F4C4520434F4D60
:100440004D414E4420343039360A4743433A203533
:100450002E342E30204156522D4C4942433A203200
:100460002E302E30204156525F415243483A20618F
:100470007672350A000A092D20436F6E736F6C6522
:10048000202D0A4553432F713A09717569740A6D1D
:100490003A096D6F7573656B65790A000A092D203D
:1004A0004D61676963202D0A443A094465627567A6
:1004B000204D65737361676520546F67676C650ACB
:1004C000583A094D617472697820446562756720F5
:1004D0004D6F646520546F67676C65202D205368ED
:1004E0006F77206B65797072657373657320696EC1
:1004F000206D617472697820677269640A4B3A09E9
:100500004B6579626F61726420446562756720543F
:100510006F67676C65202D2053686F77206B657956
:100520007072657373207265706F72740A4D3A0948
:100530004465627567204D6F75736520546F6767FA
:100540006C650A563A0956657273696F6E0A533ABA
:10055000095374617475730A433A09416374697687
:1005600061746520436F6E736F6C65204D6F6465B9
:100570000A46312D4631303A095377697463682051
:10058000746F204C6179657220302D3920284631F6
:1005900030203D204C30290A302D393A09537769F3
:1005A00074636820746F204C6179657220302D3936
:1005B0000A47524156453A09537769746368207473
:1005C0006F204C6179657220302028616C746572EF
:1005D0006E617465290A423A094A756D7020746F1C
:1005E00020426F6F746C6F616465720A4553433AC1
:1005F000094A756D7020746F20426F6F746C6F6163
:100600006465722028616C7465726E617465290A74
:10061000453A095072696E7420454550524F4D203D
:1006200053657474696E67730A4253504143453A87
:1006300009436C65617220454550524F4D0A006B6D
:1006400065796D61705F636F6E6669672E72617741
:100650003A20253032580A2E737761705F636F6ECF
:1006600074726F6C5F636170736C6F636B3A20259B
:10067000750A2E636170736C6F636B5F746F5F6379
:100680006F6E74726F6C3A2025750A2E73776170E5
:100690005F6C63746C5F6C6775693A2025750A2E10
:1006A000737761705F7263746C5F726775693A200B
:1006B00025750A2E737761705F6C616C745F6C676F
:1006C00075693A2025750A2E737761705F72616CC7
:1006D000745F726775693A2025750A2E6E6F5F67C1
:1006E00075693A2025750A2E737761705F677261AC
:1006F00076655F6573633A2025750A2E737761709E
:100700005F6261636B736C6173685F6261636B737B
:10071000706163653A2025750A2E6E6B726F3A2000
:1007200025750A0064656275675F636F6E66696749
:100730002E7261773A20253032580A2E656E61623A
:100740006C653A2025750A2E6D61747269783A20BD
:1007500025750A2E6B6579626F6172643A20257582
:100760000A2E6D6F7573653A2025750A00656563FD
:100770006F6E6669673A0A64656661756C745F6C72
:10078000617965723A2025750A003F000A6D6F7520
:1007900073653A206F66660A000A6D6F7573653A75
:1007A000206F6E0A000A6B6579626F6172643A208D
:1007B0006F66660A000A6B6579626F6172643A203F
:1007C0006F6E0A000A6D61747269783A206F66660E
:1007D0000A000A6D61747269783A206F6E0A000A25
:1007E00064656275673A206F66660A000A6465622E
:1007F00075673A206F6E0A000A0A4A756D70696E55
:100800006720746F20626F6F746C6F616465722E05
:100810002E2E2000433E2000436C656172696E6796
:1008200020454550524F4D0A000A002530325820CD
:10083000006B6579626F6172645F7265706F72746C
:100840003A20005B735D005B575D005B535D005BAE
:10085000525D005B445D005B435D000E036D006113
:10086000007900700061006400000010034B006517
:100870000079004800690076006500000004030963
:100880000409025B00030100A0FA0904000001034F
:100890000101000921110100012240000705810327
:1008A00008000109040100010300000009211101F1
:1008B0000001227B000705820320000109040200D9
:1008C0000203000000092111010001222200070596
:1008D0008303200001070503032000011201000229
:1008E00000000008484B504D010001020001063194
:1008F000FF0974A1010975150026FF0095207508F0
:1009000081020976150026FF00952075089102C026
:1009100005010902A10185020901A10005091901CA
:100920002908150025019508750181020501093086
:1009300009311581257F95027508810609381581D1
:10094000257F950175088106050C0A380215812559
:100950007F950175088106C0C005010980A1018548
:100960000319012AB700150126B7009501751081FA
:1009700000C0050C0901A101850419012AA0021576
:100980000126A002950175108100C005010906A18C
:1009900001050719E029E715002501950875018172
:1009A000029501750881010507190029FF15002628
:1009B000FF009506750881000508190129059505B0
:1009C00075019102950175039101C00011241FBEAC
:1009D000CFEFDAE0DEBFCDBF11E0A0E0B1E0ECE6A2
:1009E000F2E502C005900D92A03FB107D9F722E0D1
:1009F000A0EFB1E001C01D92A43BB207E1F70E9455
:100A0000BB160C9434290C940000FF93EF93E091F3
:100A1000F001F091F101309709F00995EF91FF9104
:100A20000895FC018591803011F0EFDFFBCF089530
:100A3000FF27E0E230E247FF0CC0419597FF09C075
:100A4000EDE26095709580959095611D711D811DF9
:100A5000911D27FF02C0219530E350E2AA27660FBF
:100A6000771F881F991FAA1FA41710F0A41B639556
:100A70005A95A9F7AA3008F0A95FA05DAF93F39546
:100A8000611571058105910541F7ED3211F4EF9380
:100A9000F395F21718F43F93F395FBCF8F91B5DFE1
:100AA000FA95E1F70895E991F9918591803021F067
:100AB000853219F0AADFF9CF089520E0E894559126
:100AC0005532C1F3503311F4689455915A3348F4B8
:100AD000505390F3220F022E220F220F200D250FCC
:100AE000F4CF0EF4219589919991533619F3533728
:100AF00029F1533559F1BC0188279927E8945C36D0
:100B000021F48991999168945591543639F446EFBE
:100B10007EF077FF0DC08FEF9FEF0AC055374AE098
:100B200039F0583540E121F0523642E009F008959D
:100B3000FF93EF937DDFEF91FF91B7CFFF93EF939B
:100B4000FC0181918030B9F360DFFBCFFF93EF931D
:100B500068DFF1CFDF93CF93CDB7DEB72596A3DF64
:100B6000CF91DF91089581E0089581E008950C947C
:100B7000B50508950C94B9051F93CF93DF9300D06A
:100B800000D01F92CDB7DEB749835A836B83309173
:100B9000F30189819A81311114C0662359F022230F
:100BA00049F00E94C30C182F682F89819A810E94F6
:100BB0006E0C03C00E94980C182F69817A81812FD6
:100BC00004C00E94C30C69817A810F900F900F902E
:100BD0000F900F90DF91CF911F910C94F813FC01AF
:100BE000262F408151816281738184810C94BC05E0
:100BF00081E00895CF93DF93EC0160E00E94EF0560
:100C0000BE01DF91CF910C94BA050C947F150C9422
:100C10007B1508950E94180B0E9409062FEF84E3AC
:100C20009CE0215080409040E1F700C000000C940F
:100C300011210F931F93CF93DF938C0161E00E94EA
:100C4000EF05EC01B8010E94B705882309F45BC0E9
:100C5000B801CE010E94F11E882309F454C0B801E6
:100C6000CE010E94D319882309F44DC0B801CE01EA
:100C70000E944D1E882309F446C0F8018281882312
:100C8000D9F1CF3D8CE5D80779F140F4C115FCE5E9
:100C9000DF0791F0C130DC4591F02EC0CC35EDE599
:100CA000DE0741F1CD35FDE5DF0709F1CB35DD4547
:100CB00019F50E945A1120C00E940A0624C0809192
:100CC0006402C82FC095C170C0FB80F98093640294
:100CD000CC2329F082E191E00E94110514C080E04C
:100CE00091E00E94110510C00E940E120CC00E94DB
:100CF000511102C00E945D11C801DF91CF911F9177
:100D00000F910C94B305C0E08C2FDF91CF911F9110
:100D10000F9108950E9446200C94B5060E94B806D3
:100D20000C944C208295982F937344E0949F9001EB
:100D300011248C7C86958695282B822F8575880FAB
:100D40002A7A2695822B089508950C94A40681E0B2
:100D500008950C94A7060895CF93C82F0E94A50666
:100D60008C2F0E94A906CF91089580E00C94AC06C8
:100D70000E944D1F0C94AC06CF930E944D1FC82FAC
:100D80008091F201C81741F1C093F2018091640291
:100D900082FF1EC080FF04C08AE291E00E9411051C
:100DA0008091640280FF0CC01F92CF9385E291E096
:100DB0009F938F930E94AA050F900F900F900F9012
:100DC0008091640280FF04C083E291E00E941105DB
:100DD0008C2FCF910C94AC06CF910895CF93DF93D5
:100DE000CDB7DEB72B970FB6F894DEBF0FBECDBFE1
:100DF0004F83588769877A878B8761110E94891092
:100E00009E012F5F3F4F86E0F90111928A95E9F725
:100E100085E0FE013796D90101900D928A95E1F7A0
:100E200089819A814C815D81452B31F09F3F31F45E
:100E300091E08F3F19F403C091E001C090E090FF72
:100E400009C049815A816B817C818D819E810E947C
:100E5000AA0F05C0C9010E94F8058111F2CF2B9697
:100E60000FB6F894DEBF0FBECDBFDF91CF910895CE
:100E7000FC01808191810E94050D0895CF93882304
:100E800009F4A9C0C82F8238C1F40E944D1F81FD0A
:100E9000A2C069E380910201909103010E941E208B
:100EA0000E94AB102FEF81EE94E0215080409040E3
:100EB000E1F700C0000069E319C0833801F50E9422
:100EC0004D1F80FD88C063E5809102019091030170
:100ED0000E941E200E94AB102FEF81EE94E0215063
:100EE00080409040E1F700C0000063E5809102017E
:100EF000909103010E942020CF910C94AB10843874
:100F0000C1F40E944D1F82FD66C067E4809102011A
:100F1000909103010E941E200E94AB102FEF81EEE2
:100F200094E0215080409040E1F700C0000067E469
:100F3000DDCF8CEF8C0F813AF8F48C2F0E94F61DD8
:100F4000811149C06C2F80910201909103010E9490
:100F5000E81F882349F06C2F8091020190910301D2
:100F60000E9420200E94AB106C2F80910201909172
:100F700003010E941E20C0CF80E28C0F883048F40D
:100F8000C77081E001C0880FCA95EAF70E946C1013
:100F9000B3CFEBE5EC0FE33040F4F0E0E95BFE4F5C
:100FA000808190E0CF910C94B01FE8E5EC0FE73121
:100FB00050F4F0E0EE0FFF1FE75EFE4F808191815D
:100FC000CF910C94C61FCD3E30F08C2F0E9440175D
:100FD000CF910C941218CF910895882309F464C01E
:100FE000823879F40E944D1F81FF5EC069E38091D1
:100FF0000201909103010E941E200E94AB1069E340
:1010000010C08338B1F40E944D1F80FF4DC063E5CE
:1010100080910201909103010E941E200E94AB105A
:1010200063E580910201909103010E9420200C94BD
:10103000AB10843879F40E944D1F82FF35C067E4FD
:1010400080910201909103010E941E200E94AB102A
:1010500067E4E7CF9CEF980F913A10F4682FE1CF47
:1010600090E2980F983050F4877091E001C0990F8A
:101070008A95EAF7892F0E947210D9CF9BE5980FC5
:10108000933020F480E090E00C94B01F98E5980F26
:10109000973120F480E090E00C94C61F8D3E20F044
:1010A0000E949B170C94121808951F93CF93DF93FF
:1010B000182FEB010E943E07209741F08FE99FE037
:1010C0000197F1F700C000002197F6CF812FDF9143
:1010D000CF911F910C94ED07893319F060E070E017
:1010E00002C060E570E00C945508882321F00E944E
:1010F0006C100C94AB100895882321F00E9472109C
:101100000C94AB100895CF92DF92EF92FF920F9361
:101110001F93CF93DF937C01D62FC72FFC01128141
:10112000058102950F700E9462108823B9F0112387
:10113000A9F08C2F807F803421F080E28D0F8830E1
:1011400068F08091980282FD09C082E00E940B1134
:101150000E94621091E0D82ED92601C0D12CCC2E4D
:10116000C2948FE0C8228C2D90E08C30910508F05D
:10117000CFC1FC01EA5AFF4F0C94CB288C2F807F03
:10118000CF70882311F0C295C07F112399F0CC2332
:1011900009F4AAC180E28D0F883010F0D11104C08B
:1011A0008C2F0E946C1003C08C2F0E947C100E9418
:1011B000AB109AC18D2F0E94ED07CC2309F4A8C172
:1011C00080E28D0F883038F1DD2329F18C2F0E94C9
:1011D000821024C08C2F807FCF70803211F0C29596
:1011E000C07FDD2319F0D130A1F13DC0809198027C
:1011F00082FF17C0112349F0CC2329F08C2F0E94C5
:101200006C100E94AB1080E070C180E00E94ED077E
:10121000CC2309F47DC18C2F0E9472100E94AB1068
:1012200077C1112371F0002341F0013031F40E94A5
:101230008C108C2B0E9494106BC10E948C108C2BF4
:101240001DC0002319F0013009F462C10E94A110F1
:1012500025C0112321F0063008F05AC10EC0053018
:1012600008F056C11BC0112361F0002331F0F701D3
:10127000858180FF39C18F7085838C2F0E9475080E
:1012800047C1002359F0D93309F03FC1FFEF07EE02
:1012900013E0F15000401040E1F735C18C2F0E945F
:1012A0007C0836C18C2F86958695837019F0813025
:1012B00061F02EC1112321F08D2F9C2F937002C05D
:1012C00080E090E00E94B01F2BC1112321F08D2FF0
:1012D0009C2F937002C080E090E00E94C61F20C146
:1012E0008D2F112319F00E94401702C00E949B17F6
:1012F0000E94121815C18C2F837009F047C011117C
:101300000BC12D2F229526952770220F220F6D2FAE
:101310006F70862F90E0A0E0B0E0022E04C0880F2E
:10132000991FAA1FBB1F0A94D2F7D4FF10C04FE029
:1013300050E060E070E004C0440F551F661F771F47
:101340002A95D2F7409550956095709503C040E07E
:1013500050E0BA01C695C695C3708A019B01082B5F
:10136000192B2A2B3B2BC901B801C23049F058F484
:10137000C13019F00E94840BCFC00E94720BCCC008
:101380000E94960BC9C00E94700BC6C0112319F0B1
:101390008C2F817001C08695882309F4BDC02D2F44
:1013A000229526952770220F220F6D2F6F70862FA2
:1013B00090E0A0E0B0E0022E04C0880F991FAA1FA1
:1013C000BB1F0A94D2F7D4FF10C04FE050E060E09A
:1013D00070E004C0440F551F661F771F2A95D2F78F
:1013E000409550956095709503C040E050E0BA017B
:1013F000C695C695C3708A019B01082B192B2A2B11
:101400003B2BC901B801C23049F058F4C13019F082
:101410000E94490C81C00E94370C7EC00E945B0C68
:101420007BC00E94AA0B78C0CF70112339F08C2F9B
:101430000E94D00B8D2F0E9475086EC08D2F0E94C8
:101440007C088C2F0E94F10B67C0D23F21F128F459
:10145000D03F41F0D13FC1F043C0D33F19F1D43F59
:1014600079F03EC0112341F0053008F051C08C2FB7
:101470008F710E94160C4CC0063008F049C0F7CF9F
:101480008091980282FF18C0112339F08C2F8F7140
:101490000E94D00B3DC01123C9F38C2F8F710E9485
:1014A000F10B36C0112329F08C2F8F710E94BB0BDA
:1014B0002FC00E94B60B2CC0112349F0CF718C2F86
:1014C0000E94D00B63E08C2F0E94F01021C081E0BD
:1014D0000E940B110230E0F082E00E940B1118C054
:1014E000112331F0002391F28D2F0E943E0710C08E
:1014F000002399F2D93349F41FEF27EE33E011505E
:1015000020403040E1F700C000008D2F0E94ED0721
:1015100088EF8C0D843020F40E944D1F0E94AC0691
:10152000DD20C9F00E945E1080FD15C0F701128217
:101530000E9458100E94D00BC7010E94CC0A0E9442
:101540005810DF91CF911F910F91FF90EF90DF9096
:10155000CF900C94F10BDF91CF911F910F91FF90E1
:10156000EF90DF90CF9008950F931F93CF93DF9369
:10157000EC01688179818A810E94100D8C010E94A2
:101580006D0C0E945E0BB801CE010E948308DF91B2
:10159000CF911F910F910895CF93DF93EC01988124
:1015A00089812B813C81232B31F08F3F31F481E005
:1015B0009F3F19F403C081E001C080E080FD1DC0A1
:1015C000CE010E941906811110C00E94621088236A
:1015D000A1F08A81882389F08091980282FD0DC054
:1015E00082E0DF91CF910C940B11CE010E94B40ADE
:1015F000CE01DF91CF910C94FA05DF91CF91089540
:1016000080E090E00E94B01F80E090E00E94C61F42
:101610000E9489100E94AB100E94C5190C941218E8
:1016200080910201909103010E9422200C94000BF2
:101630000E9479100C94100B92959F70963079F05F
:1016400010F4925001C09A50923068F4803F69F0D3
:1016500018F4883E40F409C0843F29F406C0883E4F
:1016600020F0813F11F080E0089581E00895FC01B1
:10167000808191810E94050D0E941C0B0895CF93DB
:10168000DF9300D000D01F92CDB7DEB70F900F9040
:101690000F900F900F90DF91CF910895CF93DF932C
:1016A00000D000D000D0CDB7DEB726960FB6F894A4
:1016B000DEBF0FBECDBFDF91CF910895089508958D
:1016C0000C945F0B0C94600B0E94620B60930702FA
:1016D000709308028093090290930A020C94000B05
:1016E0000C94640B0F931F93009107021091080252
:1016F0002091090230910A02602B712B822B932BCF
:101700001F910F910C94640B0F931F93009107028C
:10171000109108022091090230910A02602371237E
:10172000822393231F910F910C94640B0F931F93AB
:1017300000910702109108022091090230910A02DB
:1017400060277127822793271F910F910C94640BB8
:101750000C945F0B0E94A80B609303027093040229
:1017600080930502909306020C94000B60E070E0F9
:10177000CB010C94AA0B0F931F9341E050E060E063
:1017800070E08A019B0104C0000F111F221F331F4C
:101790008A95D2F7C901B8011F910F910C94AA0B39
:1017A0000F931F9341E050E060E070E004C0440FED
:1017B000551F661F771F8A95D2F78091030290917B
:1017C0000402A0910502B09106028A019B01082B38
:1017D000192B2A2B3B2BC901B8011F910F910C9497
:1017E000AA0B0F931F9341E050E060E070E004C04B
:1017F000440F551F661F771F8A95D2F74095509565
:10180000609570958091030290910402A091050269
:10181000B09106028A019B01082319232A233B2346
:10182000C901B8011F910F910C94AA0B0F931F933C
:1018300041E050E060E070E004C0440F551F661FB7
:10184000771F8A95D2F78091030290910402A091AC
:101850000502B09106028A019B01082719272A2751
:101860003B27C901B8011F910F910C94AA0B0F934C
:101870001F93009103021091040220910502309100
:101880000602602B712B822B932B1F910F910C94CE
:10189000AA0B0F931F930091030210910402209151
:1018A00005023091060260237123822393231F9146
:1018B0000F910C94AA0B0F931F93009103021091A8
:1018C00004022091050230910602602771278227C9
:1018D00093271F910F910C94AA0B0895990F990FBC
:1018E000890FE82FE695E695E695877051E001C0EF
:1018F000550F8A95EAF785E0E89FF0011124EC5036
:10190000FE4F20E030E070E04081CB01022E02C0AB
:10191000969587950A94E2F78170819584278523AF
:10192000842781932F5F3F4F2530310569F7089554
:10193000990F990F890F682F669566956695982F70
:10194000977085E0689FB001112440E050E080E08E
:10195000FB01E40FF51FEC50FE4F208130E0092E13
:1019600002C0369527950A94E2F721703327042E9A
:1019700001C0220F0A94EAF7822B4F5F5F4F453078
:10198000510531F70895BF92CF92DF92EF92FF9207
:101990000F931F93CF93DF938C01C0900302D090DD
:1019A0000402E0900502F0900602809107029091F7
:1019B0000802A0910902B0910A02C82AD92AEA2A8B
:1019C000FB2ACFE1D0E0D701C6010C2E04C0B695AA
:1019D000A795979587950A94D2F780FD04C0219723
:1019E00090F7B12C07C0BC2EB8018C2F0E940C14AC
:1019F0000197A9F38B2DDF91CF911F910F91FF904C
:101A0000EF90DF90CF90BF900895CF93DF93EC01DC
:101A10000E94C30CBE010E940C14DF91CF91089567
:101A20001F93CF93DF93EB019091F301992321F062
:101A3000CB010E94050D13C0882349F0CB010E9401
:101A4000C30C182F682FCE010E946E0C04C0CB016E
:101A50000E94980C182FBE01812F0E940C14DF9158
:101A6000CF911F9108951F93CF93DF93C0910B02E5
:101A700016E080910C02C81799F0D0E01C9FF0018D
:101A80001D9FF00D1124E35FFD4F40815181628164
:101A90007381848195810E944E0B2196C770E9CF96
:101AA000DF91CF911F91089540913D0250913E02E8
:101AB00060913F02709140028091410290914202F8
:101AC0000C944E0BEF92FF920F931F93CF93DF93E3
:101AD0008091420282958F7009F065C080913F022B
:101AE000882309F460C080910B02F0900C021091E1
:101AF0003D0200913E02609140027091410291E0EE
:101B00001F3F09F090E0C0910001D0910101292F01
:101B100096E0E92E8F1509F446C06115710521F094
:101B20000F3F21F030E003C031E001C0322F90E0E0
:101B300030FD36C0E89EF001E99EF00D1124DF0172
:101B4000A35FBD4F11963C911197301329C03C9172
:101B5000311326C012963C911297311121C0139671
:101B60004D915C911497461B570B4C175D07C0F4C1
:101B7000809142028F70806180934202EE5EFD4F41
:101B800080818F70806180838DE392E00E94CC0A17
:101B9000DF91CF911F910F91FF90EF900C94330D37
:101BA00001968770B7CFDF91CF911F910F91FF9072
:101BB000EF9008959F92AF92BF92CF92DF92EF92F3
:101BC000FF920F931F93CF93DF93CDB7DEB761974B
:101BD0000FB6F894DEBF0FBECDBF8C0185E0F801D3
:101BE000DE011D9601900D928A95E1F7D8011296BB
:101BF000EC9090913D02E0913E02209140023091A4
:101C000041022115310531F0EF3F31F481E09F3F72
:101C100019F403C081E001C080E0B82FB1709B2EA1
:101C200080FD47C1D8014C9111965C911197139694
:101C3000AD90BC9014978DE3C82E82E0D82EF09022
:101C40003F02B501621B730B20910001309101012D
:101C5000FF2009F4D9C0809142026217730708F08F
:101C600095C0282F207F09F052C05E1313C049137E
:101C700011C0FE2CE1100EC08F7080618093420273
:101C80000E94540DC6010E94CC0A80914202F801C4
:101C900085834DC1AB2831F05F3F31F481E04F3F88
:101CA00019F403C081E001C080E080FD03C081E041
:101CB0008E2502C080E090E0F82FF170FF2E80FFAB
:101CC0001CC080910B0220910C0236E0821709F4AF
:101CD0000BC190E0389FF001399FF00D1124E35FB4
:101CE000FD4F6181561306C06081461303C06281B7
:101CF000E61203C001968770E9CFFE2CEE2009F4AE
:101D000016C18091420281608093420254C05E13EA
:101D100006C0491304C0E11002C0F80199C0C8010F
:101D20000E94370B882361F1EE2051F1209142028D
:101D3000822F82958F7090E0029774F080913D021F
:101D400090913E0298878F831986BB86AA862C873E
:101D5000CE0107960E94CC0A86E0F801ADE3B2E01E
:101D600001900D928A95E1F70E94620D0E94540D38
:101D70000AC05E1711F1C8010E94370B81112CC0F7
:101D8000C8010E94CC0AFF24F394D1C0282F207FE1
:101D900081F77A2DB98AA88A6E2D89890E943F0B16
:101DA0008DE392E00E94CC0A86E0D6011D928A95CE
:101DB000E9F70E94540DF12CBAC04913DCCFE110B1
:101DC000DACFF8018583C8010E94CC0A86E0D601EB
:101DD0001D928A95E9F7ABC0EE2091F22091420264
:101DE000822F82958F7090E002970CF4B5CF80918E
:101DF0003D0290913E029A8389831B82BD82AC8210
:101E00002E83CE010196A6CF6217730708F044C057
:101E1000FE2CEE2009F4B4CF5E1330C049132EC05F
:101E20002091420220FD21C0822F82958F70482F81
:101E300050E041155105C9F0F80125834F30510597
:101E400041F08F5F982F9295907F822F8F70892B12
:101E50008583C8010E94CC0A86E0F801ADE3B2E0B8
:101E600001900D928A95E1F73CC086E0F801ADE360
:101E7000B2E001900D928A95E1F759C0C8010E9425
:101E8000370B811169CF80914202816080934202B9
:101E9000C8010E94CC0A4BC07A2DB98AA88A6E2D3F
:101EA00089890E943F0B86E0D6011D928A95E9F749
:101EB00018C0EE2009F464CFC8010E94370BF82E39
:101EC000882309F45DCF86E0F801ADE3B2E001902C
:101ED0000D928A95E1F78DE392E00E9438070E9407
:101EE000620D0E94540D23C04D875E878D859E85AF
:101EF0000E94050D292F22952F70223028F49F7003
:101F000039F0811105C00BC0243028F49F7049F4CA
:101F1000805E883020F0C8010E94CC0A9F2CF92CEA
:101F200006C0D80115969C91907F91F7F8CF8F2D20
:101F300061960FB6F894DEBF0FBECDBFDF91CF9193
:101F40001F910F91FF90EF90DF90CF90BF90AF90D7
:101F50009F9008951F93CF93DF93CDB7DEB72C9753
:101F60000FB6F894DEBF0FBECDBF4F835887698789
:101F70007A878B879C87CE0107960E94DA0D88238B
:101F8000D1F09F8188852A853B85232B31F08F3FB7
:101F900031F481E09F3F19F403C081E001C080E08B
:101FA00080FD47C04F81588569857A858B859C85E2
:101FB0000E944E0B3EC086E0FE013796DE01119670
:101FC00001900D928A95E1F7FF81E8856A857B850E
:101FD0006115710531F0EF3F31F481E0FF3F19F4F5
:101FE00003C081E001C080E080FD23C020910C028D
:101FF00030E0C90101968770992740910B0250E0AB
:1020000084179507F1F1F983EA837D836C8396E069
:10201000929FD001939FB00D1124A35FBD4FFE018D
:10202000319601900D929A95E1F780930C020E94EF
:10203000330D16E080910B0290910C02891771F11B
:10204000189FC0011124835F9D4F0E94DA0D8823E1
:1020500029F1E0910B021E9FF0011124E35FFD4F77
:102060004081518162817381848195810E944E0BF0
:1020700080910B0290E001968770992780930B0264
:10208000D9CF0E94180B10920C0210920B02EDE3B4
:10209000F2E086E0DF011D928A95E9F72C960FB6F3
:1020A000F894DEBF0FBECDBFDF91CF911F91089591
:1020B00080914B02859585958595089580914B0279
:1020C0008770089590914B02977081E009F480E049
:1020D000089580915602089590915602892B80931D
:1020E0005602089580959091560289238093560256
:1020F000089510925602089590915502892B80936D
:102100005502089580959091550289238093550238
:10211000089510925502089580914C0208950895F3
:102120000C948F100C9490109091980292FD08C01E
:1021300090914C02981721F080934C020C949210CD
:10214000089580914C02882329F010924C0280E07F
:102150000C9492100895CF93DF93E0910201F091D7
:102160000301809156028083E0910201F091030106
:10217000908180915502892B808380914C02882325
:1021800081F0E0910201F09103019081892B80831D
:1021900080910201909103010E94DC1F81110E9435
:1021A000A110C0910201D091030148E050E063E426
:1021B00072E0CE010E94E528892B69F088E0FE01DB
:1021C000A3E4B2E001900D928A95E1F7CE01DF9190
:1021D000CF910C94591FDF91CF9108950C948F10DB
:1021E0009091980292FD10C098E0899F900111246F
:1021F000262B20934B020E94D00B80914B02859599
:10220000859585950C94EE100C94D00B10924B0292
:1022100080E00C94EE1020914B02809582238093F5
:102220004B02982F977099F430E0482F082E000C3D
:10223000550B2417350759F09091980292FD07C06D
:102240008595859585950E94F10B0C94061108954E
:10225000CF939091980292FB222720F92817F9F04A
:10226000C82F892FC0FB82F9809398028091970232
:10227000909198020E948A1182E00E940B11809135
:10228000640280FF0CC01F92CF9385E391E09F937F
:102290008F930E94AA050F900F900F900F90CF91EF
:1022A00008958091980282FB882780F991E0892720
:1022B0000C94281181E00C94281180E00C942811D2
:1022C0006FEF7FEF80E090E00C941E2980E090E0BB
:1022D0000E94FA2821E0893E9E4F09F020E0822FDB
:1022E000089582E090E00C94F22883E090E00C9452
:1022F000F228CF9384E090E00E94F228C82F82E277
:1023000090E00E94F2282C2F30E0A901582BCA013E
:10231000CF910895CF93C92F682F84E090E00E9459
:1023200000296C2F82E290E0CF910C940029AB0140
:10233000BC018FE090E00C941229AB01BC0183E159
:1023400090E00C94122960E070E0CB010C949D1198
:1023500060E070E0CB010E9497110C94A31169EE2C
:102360007EEF80E090E00E941E2960E082E090E035
:102370000E94002960E083E090E00E940029109212
:102380000702109208021092090210920A0260E0FD
:1023900084E090E00E94002960E082E290E00E94E8
:1023A000002960E085E090E00E94002960E086E07E
:1023B00090E00E9400296FEF87E090E00E940029E2
:1023C00040E050E0BA0188E090E00E94122960E00D
:1023D0008DE090E00E94002940E050E0BA0188E1E1
:1023E00090E00E94122960E087E190E00E940029BD
:1023F00040E050E0BA018CE190E00E94122960E0D8
:1024000070E080E290E00E941E2940E050E0BA01B6
:1024100088E190E00E9412290C94A8110C94AF114D
:10242000682F8EE090E00C9400290E94D0206093E9
:1024300060027093610280936202909363026093E2
:102440005C0270935D0280935E0290935F02089538
:1024500085B7806885BF85B7806885BF089581E0AE
:1024600008950C942F1208950C9433120C94331287
:102470000C9436120C9433120C943A120C943312BE
:102480000E94281285EF92E20E94431F0E943E1292
:102490000C943C120E9434120C9433120E940015CA
:1024A0000C94AB060E94BB200E941C160E944E1288
:1024B0000C9438128F929F92AF92BF92CF92DF927C
:1024C000EF92FF920F931F93CF93DF93CDB7DEB7B9
:1024D0002A970FB6F894DEBF0FBECDBF0E9431160B
:1024E000982E81110E94151287E5A82E82E0B82E41
:1024F00000E010E0802E802F0E942415D82EF501D8
:10250000C1905F01C826B1F40F5F1F4F0530110560
:1025100089F78FEF89838A831B820E94C4208160A0
:10252000782F9D838C8349815A816B818D810E9494
:10253000EE062FC08091640281FD0E942A15E12CD5
:10254000FF24F3948C2D8F21F1F00E943112882307
:1025500099F0EE828F82DF2081E009F480E08887A5
:102560000E94C4208160782F9A8789874E815F817D
:1025700068858A850E94EE06F801E95AFD4F808140
:10258000F826F08206C0E394FF0CF4E0EF12DACFF5
:10259000BBCF81E0911001C080E02A960FB6F8947D
:1025A000DEBF0FBECDBFDF91CF911F910F91FF9086
:1025B000EF90DF90CF90BF90AF909F908F90089555
:1025C0000E945A120E94B2180C94BC06CF93DF935B
:1025D0000E941114EC01811521E5920708F045C015
:1025E000811530E5930708F094C0883E910528F5E1
:1025F000803E910508F0F8C0883A910570F4853A5C
:10260000910508F07CC08130910509F475C008F48B
:10261000E8C0049708F0E8C0E4C08F3B910508F0DB
:10262000E0C0C85AD0E0CC0FDD1FC65BDE4F09907A
:10263000D881C02DCE019464D8C0811540E29407A2
:1026400058F4811551E0950708F0CEC08D3E9105F4
:1026500008F4C7C09065C9C0C11580E4D80708F464
:10266000C0C0DF70CE01906AC0C0811525E5920719
:10267000A8F4811534E5930708F095C0811543E56A
:10268000940708F07BC0811552E5950708F061C0FA
:10269000D82FCC27CE01816F906AA7C0C11589E5DC
:1026A000D807A0F4C11528E5D20708F082C0C115EB
:1026B00036E5D30708F095C08C2F0E94A5148F71C2
:1026C00090E0D82FCC27CE0190628FC0C1154AE58B
:1026D000D40708F474C0CE0190568115904208F0DA
:1026E00080C08D2F8F710E94A514DD27D0628F715D
:1026F000AE01582BCA0179C081E090E076C0C55A7E
:10270000D0E0C858DE4F8881C82FD0E0CE01906459
:102710006CC074E0969587957A95E1F7282F237021
:102720003C2F337081E090E002C0880F991F3A95EA
:10273000E2F79C68AC01522B9A019C2F9F709695F2
:10274000969550E2959FE0011124C9018C2B9D2B99
:102750004CC08370992721E030E002C0220F331F64
:102760008A95E2F79C2F9695969580E2989FE001D6
:102770001124C22BD32BCE019C6837C083709927BC
:1027800021E030E002C0220F331F8A95E2F79C2F30
:102790009695969540E2949FE0011124C22BD32B8D
:1027A000CE019A6822C0D82FCC27CE01846F906AC0
:1027B0001CC0DC2FCC27CE01806F906A16C08C2FF6
:1027C0008F700E94A51494E0D695C7959A95E1F76D
:1027D000CF70D0E0DC2FCC27D0699E01282BC90117
:1027E00004C080E090E001C0CE01DF91CF91089558
:1027F000E72FF0E095E0899FE00DF11D1124EE0F29
:10280000FF1FEE0FFF1FE60FF11DEE0FFF1FE85237
:10281000FF4F8591949108950E94F8130E94E6124B
:1028200008958238910569F1B0F48133910509F476
:102830006DC048F48932910509F463C08A3291056C
:1028400009F469C008958533910509F455C08933A9
:102850009105B9F00895833E910569F138F4803E01
:102860009105B1F0823E910509F10895863E9105EA
:10287000A9F1873E9105B9F1843E910509F064C044
:1028800023C02091970220FD4FC021FD4DC0089527
:102890008091970280FD44C08091980280FF44C0DF
:1028A0008091970284FD42C083EE4DC080919702D3
:1028B00082FF38C0F5CF8091970282FD33C08091AE
:1028C000980280FD31C0ECCF8091980281FF32C028
:1028D0008091970284FD2AC087EE35C080919702CF
:1028E00083FF26C0F5CF8091970283FD21C08091A0
:1028F000980281FD1FC0ECCF8091970285FD1CC01E
:102900001DC08091970285FD19C016C08091970265
:1029100086FD16C017C08091970286FD13C010C0B7
:1029200089E311C082EE0FC080EE0DC080E00BC0C5
:1029300086EE09C084EE07C089E205C085E303C0C6
:102940008AE201C081E390E008959091970292FF9E
:102950000DC0282F2871283019F4877F846006C0A5
:10296000282F2471243011F48B7F886093FF0DC0D1
:10297000282F2871283119F4877E846106C0282FFA
:102980002471243111F48B7E88612091980220FFFC
:102990000DC0382F3871383019F4877F816006C038
:1029A000382F3171313011F48E7F886021FF0DC0D6
:1029B000282F2871283119F4877E816106C0282FBD
:1029C0002171213111F48E7E886194FD877E0895F6
:1029D0000C9460110E9431168FE39CE90197F1F786
:1029E00000C000000E94311680E00E94241580FF84
:1029F00004C00E94E8140C94112108950C94EA1468
:102A00000E946611811102C00E940E120E94711173
:102A1000809364020E9479119093980280939702A8
:102A20000E94FE140E947511682F70E080E090E013
:102A30000E94700B60910302709104028091050264
:102A4000909106020C94A80BE82FF0E0E256FD4F9F
:102A500080810895CF92DF92EF92FF920F931F93A0
:102A6000CF93DF9389E591E00E9411058EE9E82E6E
:102A700082E0F82EC0E0D0E094E5C92E91E0D92E96
:102A80000CE411E0DF93CF93DF92CF920E94AA056E
:102A900081E591E00E941105F70181917F010E947B
:102AA00092061F928F931F930F930E94AA058AE4A8
:102AB00091E00E94110521968DB79EB708960FB63A
:102AC000F8949EBF0FBE8DBFC530D105D9F6DF91FA
:102AD000CF911F910F91FF90EF90DF90CF900895CD
:102AE00080EA8A95F1F7089500C008950C94701556
:102AF00008950C9478150C9479150C9478150C9411
:102B00007D15F894E82FE295EF70F0E031A1282FC1
:102B10002F7081E090E001C0880F2A95EAF7982F86
:102B20009095932391A392A1892B82A378940895E1
:102B30000F931F93CF93DF93CFE7D1E089918F3F1E
:102B400011F00E94811581E0C438D807B9F7CBE7AE
:102B5000D1E00FE711E089918F3F11F00E948115BC
:102B60000C171D07C1F7DF91CF911F910F910895A9
:102B7000CF92DF92EF92FF920F931F93CF93DF9349
:102B80008C01C62FD0E0CE0181589E4F7C01FC0104
:102B900090819F3F09F447C0D62EF894E92FE29523
:102BA000EF70F0E081A19F7021E030E001C0220FC2
:102BB0009A95EAF7822B81A382A12095282322A34C
:102BC00078940E947415EBE7F1E04FE751E031E0B3
:102BD000C12C21912F3F89F0A22FA295AF70B0E0B8
:102BE00090968C9190E02F7002C0959587952A95CC
:102BF000E2F780FD02C0832F01C080E0C82A330FB6
:102C00004E175F0731F7F70180818F3F11F00E9467
:102C1000811561E0C11001C060E08D2D0E94761524
:102C2000C00FD11FC882DF91CF911F910F91FF90EC
:102C3000EF90DF90CF9008950E94981585E0EEE91F
:102C4000F2E0DF01982F1D929A95E9F7E9E9F2E0A9
:102C5000DF011D928A95E9F785E00E9478160C94B1
:102C60000506FF920F931F93CF93DF9300D000D000
:102C70001F92CDB7DEB78E010F5F1F4F85E0F801C1
:102C800011928A95E9F7F12C6F2DC8010E94B815B1
:102C9000F394F5E0FF12F8CF45E050E0B80189E980
:102CA00092E00E94E528FF24F394009709F4F12CA8
:102CB000892B41F085E0F801A9E9B2E001900D927D
:102CC0008A95E1F72F2D45E06EE972E089E992E0FF
:102CD0000E9479160E9407068F2D0F900F900F907B
:102CE0000F900F90DF91CF911F910F91FF9008955A
:102CF0000895FF920F931F93CF93DF938C01F62ECD
:102D0000D72FC42F222349F081E0809367020E94CD
:102D1000C4209093660280936502809167028823A5
:102D2000C1F080916502909166020E94DC200597B7
:102D300080F0EF2DFD2FD8014C2F50E0CD01801BEE
:102D4000910B841795071CF48D918193F7CF109206
:102D50006702DF91CF911F910F91FF9008950E941C
:102D600071230E9452120C947D230E9481230E94A1
:102D7000E0120C949F230E9462200E9458230E941C
:102D800040120E94AF160E94B5160E944A12FBCF55
:102D900080916E0280FF06C06091090170E0660FAD
:102DA000771F26C081FF04C06091090184E005C03F
:102DB00082FF07C06091090188E0689FB00111247B
:102DC00017C090916D029923D1F060910801961778
:102DD00088F72091090188E0289F90011124929F93
:102DE000A001939F500D112470E0CA010E94B728E2
:102DF0006038710540F46115710519F406C068E08A
:102E000070E0862F08958FE7089581E008958091FE
:102E10006E0280FF08C06091050170E075956795AE
:102E20007595679521C081FF06C06091050170E02E
:102E30007595679519C082FF04C06091050170E027
:102E400010C090916C02992399F06091040196173B
:102E5000A0F780910501899FC001112470E00E94B4
:102E6000B7286038710540F46115710519F406C082
:102E700061E070E0862F08958FE7089581E008955E
:102E80008D3E21F40E94C816819504C08E3E29F41F
:102E90000E94C8168093720208958F3E21F40E940A
:102EA000C816819504C0803F29F40E94C8168093FB
:102EB00071020895893F19F40E94071705C08A3FDF
:102EC00031F40E94071781958093730208958B3F18
:102ED00021F40E940717819504C08C3F29F40E94B9
:102EE00007178093740208959FE0980F983078F444
:102EF00021E030E0A90102C0440F551F9A95E2F786
:102F0000CA0190917002892B8093700208958D3FC1
:102F100021F480916E0281600BC08E3F21F480917C
:102F20006E02826005C08F3F29F480916E0284603A
:102F300080936E0208958D3E39F49091720297FF4E
:102F400035C01092720259C08E3E29F490917202DF
:102F50001916BCF32BC0909171028F3E29F497FF94
:102F600025C01092710249C0803F19F41916CCF3A4
:102F70001DC090917302893F29F41916BCF4109278
:102F800073023BC08A3F19F497FF10C0F8CF8B3F04
:102F900039F49091740297FF09C0109274022DC009
:102FA0008C3F21F4909174021916BCF39FE0980FA6
:102FB000983080F421E030E0A90102C0440F551F91
:102FC0009A95E2F7CA0180959091700289238093C7
:102FD000700213C08D3F21F480916E028E7F0BC072
:102FE0008E3F21F480916E028D7F05C08F3F29F4C2
:102FF00080916E028B7F80936E02809171028111AD
:1030000006C080917202811102C010926D028091FF
:103010007302811106C080917402811102C0109266
:103020006C0208958091640283FF7EC08FE891E076
:103030000E941105809170021F928F938AE891E09F
:103040009F938F930E94AA0588E891E00E94110542
:1030500080917102282F082E000C330B3F938F9321
:1030600085E891E09F938F930E94AA0583E891E001
:103070000E94110580917202282F082E000C330B3C
:103080003F938F9380E891E09F938F930E94AA05CE
:103090008EE791E00E94110580917302282F082E7F
:1030A000000C330B3F938F938BE791E09F938F93AB
:1030B0000E94AA0589E791E00E941105809174029F
:1030C000282F082E000C330B3F938F9386E791E057
:1030D0009F938F930E94AA0583E791E00E941105B8
:1030E00080916D021F928F9380E791E09F938F9361
:1030F0000E94AA058EE691E00E94110580916E0261
:103100001F928F938BE691E09F938F930E94AA0565
:1031100088E691E00E9411058DB79EB74C960FB6D8
:10312000F8949EBF0FBE8DBF0E94C42020917102F3
:10313000211104C020917202222321F090936B028E
:1031400080936A0220917302211104C020917402BD
:10315000222321F090936902809368028FE692E027
:103160000C94A21FEF92FF920F931F93CF93DF93C4
:1031700000D000D000D0CDB7DEB786E0EFE6F2E0B9
:10318000DE01119601900D928A95E1F7E0907102AF
:10319000F090720200917302109174021092710209
:1031A000109272021092730210927402E11003C026
:1031B000FF2009F45DC080916A0290916B020E9429
:1031C000DC20AC0190916D02992339F020910A0125
:1031D00030E02417350758F04BC020910B018AE0EE
:1031E000289F900111242417350718F041C09F3FF4
:1031F00019F09F5F90936D02EE2061F00E94C81657
:103200001E1414F09FEF01C091E0989F902D11249F
:1032100090937102FF2061F00E94C8161F1414F0F1
:103220009FEF01C091E0989F902D1124909372021E
:10323000309171023323E1F0209172022223C1F018
:1032400045EB3403C0011124992319F090937102C6
:1032500003C081E08093710235EB2303C001112488
:10326000992319F09093720203C081E08093720257
:10327000011103C0112309F45DC08091680290918F
:1032800069020E94DC20AC0190916C02992339F014
:103290002091060130E02417350758F04BC02091EB
:1032A00007018AE0289F900111242417350718F0A0
:1032B00041C09F3F19F09F5F90936C02002361F023
:1032C0000E940717101614F09FEF01C091E0989F1D
:1032D000902D112490937302112361F00E9407171F
:1032E000111614F09FEF01C091E0989F902D1124CA
:1032F00090937402309173023323E1F020917402B1
:103300002223C1F045EB3403C0011124992319F0A5
:103310009093730203C081E08093730235EB230323
:10332000C0011124992319F09093740203C081E025
:10333000809374028091710281110BC0809172029E
:10334000811107C080917302811103C080917402C2
:1033500081110E941218EB82FC820D831E8386E08D
:10336000FE013196AFE6B2E001900D928A95E1F749
:1033700026960FB6F894DEBF0FBECDBFDF91CF917A
:103380001F910F91FF90EF900895EFE6F2E086E035
:10339000DF011D928A95E9F710926D0210926C027E
:1033A00010926E020895CF93DF93EC01FB018281AE
:1033B000882309F43CC1C430FDE5DF0760F4CB3F4E
:1033C0009CE5D90788F49E0122503C452431310503
:1033D00008F02EC109C0C236EDE5DE0729F0C63A75
:1033E000FDE5DF0709F024C10E947911909398024E
:1033F00080939702C1318CE5D80709F4C6C008F064
:1034000042C0C930ECE5DE0709F49BC000F5C530C9
:103410008CE5D80709F485C078F4C330ECE5DE0705
:1034200009F478C008F07AC0C230DC4509F0F5C074
:10343000809197028160EFC0C7309CE5D90709F4FD
:1034400078C008F07AC0809197028061E4C0CD30E6
:10345000FCE5DF0709F487C058F4CB309CE5D907B9
:1034600009F479C008F07BC08091970288606FC032
:10347000CF30FCE5DF0709F480C008F082C08091FE
:103480009702877FC8C0CE3F9CE5D90709F471C079
:1034900000F5C531FCE5DF0709F485C068F4C331E8
:1034A0009CE5D90709F475C008F095C00E94180B77
:1034B000809197028F77AFC0CC3FFCE5DF07A9F181
:1034C00008F054C0CB3FDC4509F0A7C080919802BA
:1034D00040C0C230EDE5DE0709F489C058F4C115DB
:1034E0008DE5D80709F45AC008F069C080919802A8
:1034F00082602FC0C236EDE5DE0709F47CC0C63A13
:10350000FDE5DF0709F481C0C330DD4509F085C062
:1035100080E06EC08091970282607DC080919702AA
:1035200016C080919702886076C080919802826070
:103530004FC08091970280626EC080919702806434
:103540006AC00E94180B80919702806864C08460F2
:1035500062C081603DC0809197028E7F5CC0809187
:1035600097028D7F58C08091970216C08091980273
:1035700018C0809198028D7F2BC0809197028F7E1A
:103580004AC0809197028F7D46C0809197028F7BC1
:1035900042C080919702877F8B7F3DC080919802C7
:1035A0008D7F8E7F15C08091970282FB222720F9A4
:1035B00091E0922790FB82F990FB83F92CC08091D7
:1035C0009802982F909591708E7F892B90FB81F9AE
:1035D0008093980222C00E94180B8091970287FB6B
:1035E000222720F991E0922790FB87F914C081E00F
:1035F0000E94101212C08091970284FB222720F9AA
:1036000091E0922790FB84F906C080919702982F51
:10361000909590FB80F9809397028091970290910A
:1036200098020E948A110E94180B80E001C081E07C
:10363000DF91CF910895809104011F928F93809123
:1036400005011F928F93809108011F928F938091A3
:1036500009011F928F9380910A011F928F9380918D
:103660000B011F928F9382EB91E09F938F930E94A7
:10367000AA058DB79EB70E960FB6F8949EBF0FBEE3
:103680008DBF0895883220F58E3108F068C08B30E8
:1036900091F1C0F4873009F0BEC081E080930B0146
:1036A00084E180930A018AE0809309018EE180938E
:1036B000080188E08093050188E28093040184E199
:1036C00093E0C6C0833109F443C0843169F1A3C0DB
:1036D0008F3409F49EC028F4893231F1883359F0CF
:1036E0009AC0813531F008F4D4C0823509F4A7C0FE
:1036F00092C08FEFA5C086E393E00E9411050E945F
:103700001B1B1F9281E08F931F9288E08F938FE2A3
:1037100092E09F938F930E94AA050F900F900F90B5
:103720000F900F900F9096C083E393E00E941105D5
:1037300080917902882309F4AAC01092790210922C
:103740007802109277021092760210927502B1C040
:1037500085E293E00E9411050E941B1B7BC08D51E6
:1037600080937902833031F170F48130D1F082306E
:1037700009F03FC08AE091E090937802809377024D
:1037800081E991E01FC0853059F108F1863089F553
:1037900084E091E090937802809377028CEC91E042
:1037A00011C08BE091E0909378028093770288E8D3
:1037B00091E008C089E091E09093780280937702CD
:1037C0008DE991E0909376028093750218C088E0AD
:1037D00091E090937802809377028AEA91E0F2CFA9
:1037E00085E091E0909378028093770289EB91E0F5
:1037F000E9CF1092790282E293E00E941105809154
:103800007902882309F455C01F928F938EE193E0CB
:103810000DC08AE015C081E193E01AC097FF47C050
:10382000108280811F928F938BE093E09F938F9300
:103830000E94AA050F900F900F900F900BC081E08F
:10384000E0917702F0917802309729F588E093E0D3
:103850000E94110520917902222359F1809175026D
:1038600090917602009711F484E891E09F938F93F2
:103870001F922F938FEF92E09F938F930E94AA0540
:103880000F900F900F900F900F900F9016C080E048
:10389000089586EFD5CF2081082E000C990B820F5A
:1038A000911D8F3F910509F00CF4B8CF8FEF808305
:1038B000B8CF8BEF92E00E94110581E00895CF937D
:1038C000C82F1F928F938CE493E09F938F930E9455
:1038D000AA0581E090E0A0E0B0E0BC01CD0104C009
:1038E000660F771F881F991FCA95D2F70E94700B29
:1038F0000F900F900F900F90CF910C94180BEF92A8
:10390000FF920F931F93CF93DF938B3109F4EDC098
:1039100008F08EC08B3009F4B1C008F078C0863052
:1039200009F4AFC020F4853009F4BDC04EC1873022
:1039300009F4C0C0883009F048C10E9475111F9277
:103940008F938DE697E09F938F930E94AA050E9424
:10395000711183FB992790F91F929F9382FB9927FE
:1039600090F91F929F9381FB992790F91F929F9343
:10397000982F91701F929F931F928F9384E297E0EC
:103980009F938F930E94AA050E94791187FB22279B
:1039900020F91F922F9386FB222720F91F922F9345
:1039A00085FB222720F91F922F9384FB222720F9E1
:1039B0001F922F9383FB222720F91F922F9382FBC4
:1039C000222720F91F922F9391FB222720F91F9283
:1039D0002F93292F21701F922F9381FB222720F9EB
:1039E0001F922F93282F21701F922F939F938F93B5
:1039F0008FE396E09F938F930E94AA058DB79EB7A1
:103A000088960FB6F8949EBF0FBE8DBF35C080312B
:103A100009F495C020F48E3009F47BC0D6C08631FD
:103A200009F4A8C0893109F0D0C08CEB93E084C0C0
:103A30008A32E1F060F4873209F4C3C028F48E3191
:103A400008F4C3C08D51BEC0893269F1BEC0833451
:103A500048F48A3308F0B3C0853309F4B2C0883320
:103A600069F0B3C0833409F4ACC0AFC088E198E01A
:103A70000E9411050E940E12C1E0ACC08CE994E0D6
:103A80005BC080916402817F8E7F8093640285E7B2
:103A900094E00E94110584E198E00E94110581E004
:103AA00080937A02E9CF88EF97E00E9411050E9487
:103AB0000A06E2CF80916402C82FC095C170C0FB96
:103AC00080F980936402CC2329F08CEE97E00E9469
:103AD000110580C08FED97E00E941105809164026E
:103AE000897F877F80936402C7CF9091640291FBA6
:103AF000CC27C0F981E0C827892FC0FB81F98093CA
:103B00006402CC2319F082ED97E029C084EC97E0A1
:103B100013C09091640292FBCC27C0F981E0C827C2
:103B2000892FC0FB82F980936402CC2319F085EBC6
:103B300097E015C085EA97E00E9411059DCF90910E
:103B4000640293FBCC27C0F981E0C827892FC0FB12
:103B500083F980936402CC2351F089E997E00E94B5
:103B600011058091640281608093640233C08CE807
:103B700097E0E2CF0E94D020162F072FF82EE92ED3
:103B8000D0919602C09118010E944D1FEF92FF92B2
:103B90000F931F931F92DF931F92CF931F928F93C8
:103BA00081E593E09F938F930E94AA058DB79EB7FE
:103BB0000C960FB6F8949EBF0FBE8DBF5DCF895394
:103BC00001C080E00E945F1C57CF8AE897E00E9406
:103BD0001105C0E08C2FDF91CF911F910F91FF90C5
:103BE000EF90089580E008950C94F21DCF93C82FB4
:103BF00080917A02813071F040F0823009F045C046
:103C00008C2F0E94421B81E046C00E9469108232C4
:103C1000F1F504C00E946910823261F48C2F0E9479
:103C2000F41D811104C08C2F0E947F1C2CC081E0E8
:103C300090E029C08C2F0E94F21D811123C0C43155
:103C4000C9F058F4CB3069F0C031B9F482E0809308
:103C50007A0288E30E94421B15C0C93259F0C8336A
:103C600061F485E794E00E94110588E493E00E94E6
:103C7000110508C010927A020CC086E493E00E94FD
:103C8000110507C081E0817006C010927A0280E0C1
:103C900002C080E0F8CFCF910895CF93DF938631B3
:103CA0009C4541F5EB010E946910982F8A81209173
:103CB000020130910301882379F09A7A81E009F4B6
:103CC00080E080937B02911102C069E201C065E34C
:103CD000C9010E941E200AC080917B02811102C08E
:103CE00069E201C065E3C9010E9420200E94AB1077
:103CF00080E001C081E0DF91CF9108950F931F9381
:103D0000CF93DF93C42FD22FFC0182818823C9F087
:103D100040937E020E94C42090937D0280937C0297
:103D200080E28C0F883008F057C0C77081E001C076
:103D3000880FCA95EAF7DF91CF911F910F910C94EC
:103D4000750880917E02481330C080917C0290916A
:103D50007D020E94DC20883C910538F510E21D0FA1
:103D6000CD17B9F080E28C0F883040F4C77081E045
:103D700001C0880FCA95EAF70E947C08183028F520
:103D800081E09D2F977001C0880F9A95EAF70E94F5
:103D90007508802F0E946C081830F0F4D77081E00D
:103DA00001C0880FDA95EAF70AC080E28C0F8830EC
:103DB00098F4C77081E001C0880FCA95EAF7DF91D7
:103DC000CF911F910F910C947C08802FDF91CF91A0
:103DD0001F910F910C946C08DF91CF911F910F915F
:103DE00008950F939C01CB01243F4CE5340731F13A
:103DF00088F4293DFCE53F07D9F02A3D4CE534071E
:103E000079F1283D3C45A9F506E221EE41EE68ED49
:103E10007CE52BC0263FFCE53F07E1F0A8F0273FFB
:103E20003C4539F507E225EE46EE67EF7CE51DC01F
:103E300007E225EE45EE69ED7CE517C006E221EECE
:103E400040EE64EF7CE511C007E225EE44EE65EF3D
:103E50007CE50BC006E221EE42EE66EF7CE505C094
:103E600008E221E045EE6AED7CE50E947E1E80E0DE
:103E700008C0FC018281882319F010927E0201C0E3
:103E800081E00F9108959093F1018093F0010895DE
:103E900090938402809383020895E0918302F091CD
:103EA0008402309721F00190F081E02D099480E0A8
:103EB0000895EF92FF920F931F93CF93DF93E091BA
:103EC0008302F09184023097B1F18C010280F3817A
:103ED000E02D09958091640282FF2DC080FF04C00F
:103EE00081E398E00E941105E80118E08BE2E82EDA
:103EF00088E0F82E8091640280FF0BC088811F92B9
:103F00008F93FF92EF920E94AA050F900F900F904F
:103F10000F90115021961111EDCF8091640280FF16
:103F20000AC089E298E0DF91CF911F910F91FF9035
:103F3000EF900C941105DF91CF911F910F91FF909D
:103F4000EF900895E0918302F0918402309739F068
:103F500022E0DC012C930480F581E02D0994089582
:103F600020918102309182022817390771F09093D5
:103F7000820280938102E0918302F0918402309763
:103F800021F00680F781E02D0994089520917F02A9
:103F9000309180022817390771F090938002809346
:103FA0007F02E0918302F0918402309721F0008437
:103FB000F185E02D09940895FC01329697E080E0A8
:103FC000915029F021912223D9F38F5FF9CF0895E1
:103FD000662349F0FC01329608962191621729F078
:103FE000E817F907D1F780E0089581E008959C0172
:103FF000FC0132969FEF80E04191461789F09F3F88
:1040000019F4411101C0982F8F5F8630A9F79F3FA7
:1040100039F0F901E90FF11D97FDFA9562830895D2
:1040200008959C012A5F3F4FFC014281461301C065
:104030001282019682179307B9F708950C94F71F1F
:104040000C941120029626E0FC0111922A95E9F7C2
:10405000089508950C94292083E0809385020C94A0
:104060002A20811102C081E001C082E08093850294
:104070000C942A200C94312081E0809385020C94CA
:104080002A200C943C2008950C9443200C94442046
:104090000C9443200C9443200C944320CF930E9413
:1040A0004A200E9431160E944820C0E08C2F0E94B6
:1040B0002415811104C0CF5FC530C1F701C081E074
:1040C000CF91089508951F920F920FB60F92112469
:1040D0008F939F93AF93BF9380918602811113C0FA
:1040E0008091A3029091A402A091A502B091A60292
:1040F0004196A11DB11D8093A3029093A402A093A9
:10410000A502B093A602BF91AF919F918F910F909E
:104110000FBE0F901F9018958091AB02843031F143
:104120000E948A061092860220E488E190E00FB691
:10413000F894A895809360000FBE2093600083B729
:10414000817F846083BF83B7816083BF78948895C3
:1041500083B78E7F83BF0FB6F894A89580916000D7
:10416000886180936000109260000FBE08950E94E5
:10417000180B0C948E0682E084BD93E095BD9AEFF7
:1041800097BD80936E0008952FB7F8948091A30295
:104190009091A402A091A502B091A6022FBF08950C
:1041A0002FB7F8946091A3027091A4028091A502A8
:1041B0009091A6022FBF08959C014FB7F89480916B
:1041C000A3029091A402A091A502B091A6024FBFB4
:1041D000821B930B089578941F920F920FB60F9243
:1041E00011248F939F93AF93BF938091A3029091DB
:1041F000A402A091A502B091A6020196A11DB11D35
:104200008093A3029093A402A093A502B093A60268
:10421000BF91AF919F918F910F900FBE0F901F9004
:10422000189587E797E790930108809300089AE034
:1042300088E10FB6F894A895809360000FBE909324
:104240006000FFCF809195020895089522E02093A9
:10425000E9002FEF3091E800215035FD06C035ED23
:104260003A95F1F700002111F5CF2091E80025FFE4
:104270000BC040E050E066E070E00E940E248091A8
:10428000E8008E778093E8000895CF93DF9321E0D4
:104290002093E9002FEF3091E800215035FD06C052
:1042A00035ED3A95F1F700002111F5CF2091E800A6
:1042B00025FF14C0EC0140E050E068E070E00E948F
:1042C0000E248091E8008E778093E80088E0FE015C
:1042D000ADE8B2E001900D928A95E1F7DF91CF91C0
:1042E00008958093890270938B0260938A02809173
:1042F000AB02843001F582E08093E9008FEF90916A
:10430000E800815095FD06C095ED9A95F1F7000003
:104310008111F5CF8091E80085FF0DC040E050E0AD
:1043200063E070E089E892E00E940E248091E8004A
:104330008E778093E8000895BC0184E00C9471218D
:10434000BC0183E00C94712187E598E00E9411057F
:104350008091AA02811109C00E949F250E94FC251C
:104360008091E20084608093E200089583E598E004
:104370000E9411051092AA0208958FE498E00E940D
:1043800011050C9441208BE498E00E941105609186
:10439000A70281E0611101C080E00C942C2087E429
:1043A00098E00E9411059091AB0281E0943009F0F1
:1043B00080E06091A7020C943120209188022F5F49
:1043C000822F62E30E94AB28992319F02093880280
:1043D00008951092880280918C02882371F1809157
:1043E000AB02843041F58091E9008F702091EC00A0
:1043F000922F917020FD90E8892B93E09093E90033
:104400009091EB0090FF14C09091EE0097FF10C0C8
:104410009091E80095FF03C01092F100F9CF9091C0
:10442000E80090FF05C09091E8009E779093E80027
:104430008F708093E90010928C02089542E061EC45
:1044400081E00E94182542E261EC82E00E9418257A
:1044500042E261EC83E00E9418259091AB0281E07A
:10446000943009F080E06091A7020C943A2080918A
:10447000AD02833009F461C030F4813071F08230D4
:1044800009F49AC008958A3009F486C08B3009F483
:104490006CC0893009F0A8C020C08091AC02813A7C
:1044A00009F0A2C08091E800877F8093E8008091A6
:1044B000B0029091B102892B21F468E08DE892E07E
:1044C00003C060E080E090E070E00E945924809199
:1044D000E8008B778093E80008958091AC028132E8
:1044E00009F082C08091B0029091B102029708F069
:1044F0007BC08091E800877F8093E8008091E8008E
:1045000082FD05C08091AB028111F8CF6DC0209172
:10451000F3008091F20090E0922B029731F48091A9
:10452000F100813011F0863021F48091F100809308
:1045300095028091E8008B7753C08091AC02813A5C
:1045400009F052C08091B0029091B102892B09F01C
:104550004BC08091E800877F8093E8008091E8005D
:1045600080FFFCCF8091180136C08091AC0281326F
:10457000D9F58091B0029091B102892BA9F5809173
:10458000E800877F8093E8000E944D258091AE026D
:10459000809318010C94180B8091AC02813221F5A4
:1045A0008091E800877F8093E8000E944D258091EC
:1045B000AF028093960208958091AC02813AA1F4F3
:1045C0008091E800877F8093E8008091E80080FF79
:1045D000FCCF809196028093F1008091E8008E7765
:1045E0008093E8000C944D2508959FB7F89410929D
:1045F0008C029FBF9091AB02943009F057C090910C
:10460000E9009F703091EC00232F217030FD20E8ED
:10461000922B23E02093E9002091EB0020FF43C080
:104620002091EE0027FF3FC020918702222321F036
:104630002091E80025FF37C01092870226E03091D4
:10464000E80035FD15C03091AB02343061F5309192
:10465000EB0035FD28C0215021F481E080938702D2
:1046600022C0EFE9FFE03197F1F700C00000E7CF8B
:104670008093F1008091E80085FD0AC08091E800F8
:1046800080FFFCCF8091E8008E778093E80006C021
:104690008FB7F89421E020938C028FBF9F70909386
:1046A000E90080E008959F709093E9008FEF0895EE
:1046B00084B7877F84BF0FB6F894A8958091600077
:1046C000886180936000109260000FBE90E080E8E7
:1046D0000FB6F89480936100909361000FBE0C9424
:1046E0003C200E949F250E94FC25E2EEF0E08081A4
:1046F0008460808378940C9490288CE091E00C94F2
:10470000481F8091AB028530C9F483E498E00E9491
:1047100011058091AB02853079F40E948C20809144
:10472000A9028823B1F30E944E20882391F30E94AE
:10473000F8230E94180BEDCF0C94B720089508952C
:104740000C94A223292F332723303105C9F060F4BC
:104750002130310581F02230310509F041C08BE56F
:1047600090E021E838E040C021323105E1F022320A
:10477000310531F135C082E190E02CED38E034C0F4
:1047800099278130910549F028F0029749F5EBE52A
:10479000F8E005C0EDE7F8E002C0EBE6F8E0849150
:1047A00090E09F0121C063307105D0F4660F771F40
:1047B000FB01E651FE4F2081318189E090E014C079
:1047C0006330710568F4FB01EE0FFF1FEC51FE4FE3
:1047D00020813181FB01EF51FE4F808190E004C0C8
:1047E00080E090E020E030E0FA01318320830895FA
:1047F00080E189BD82E189BD09B400FEFDCF8091D1
:10480000D8008F7D8093D8008091E00082608093F3
:10481000E0008091E00081FDFCCF0895CF92DF920F
:10482000EF92FF920F931F93CF93DF93EC018B01D5
:104830007A010E946C25811133C0E114F10439F032
:10484000F70180819181081B190BC80FD91FC12C5A
:10485000D12C0115110519F18091E80085FD16C0D4
:104860008091E8008E778093E800E114F10449F02C
:10487000F70180819181C80ED91ED182C08285E066
:104880000FC00E946C25882321F30AC08991809370
:10489000F10001501109FFEFCF1ADF0ADACF80E0F3
:1048A000DF91CF911F910F91FF90EF90DF90CF900C
:1048B00008952091B2023091B3022617370748F0CD
:1048C0006115710539F42091E8002E772093E800F6
:1048D00001C0B901FC0120E06115710579F18091F9
:1048E000AB028823F1F18530F1F18091E80083FD7E
:1048F0003CC08091E80082FD2EC08091E80080FFDE
:10490000EBCF2091F3008091F20090E0922B6115A3
:10491000710551F08830910538F421912093F10010
:10492000615071090196F3CF21E0089709F020E06A
:104930008091E8008E778093E800CECF2111CFCF11
:104940000AC08091AB02882361F0853061F08091CC
:10495000E80083FD0AC08091E80082FFF2CF80E08A
:10496000089582E0089583E0089581E008952091FC
:10497000B2023091B3022617370748F0611571056E
:1049800039F42091E8002E772093E80001C0B901A6
:10499000FC0120E06115710591F18091AB02882343
:1049A00009F440C0853009F43FC08091E80083FDE0
:1049B0003DC08091E80082FD2FC08091E80080FF1B
:1049C000E9CF2091F3008091F20090E0922B6115E5
:1049D000710559F08830910540F424912093F1003D
:1049E0003196615071090196F2CF21E0089709F0E4
:1049F00020E08091E8008E778093E800CBCF2111F2
:104A0000CCCF0AC08091AB02882361F0853061F081
:104A10008091E80083FD0AC08091E80082FFF2CF18
:104A200080E0089582E0089583E0089581E008958C
:104A3000982F973068F59093E900981739F07091A6
:104A4000EC002091ED005091F00003C0242F762F50
:104A500050E021FD02C09F5FECCF3091EB003E7F24
:104A60003093EB003091ED003D7F3093ED003091BD
:104A7000EB0031603093EB007093EC002093ED007D
:104A80005093F0002091EE0027FDE5CF80E00895DF
:104A90008F708093E90081E008958091AC0287FFD8
:104AA00011C08091E80082FD05C08091AB028111A8
:104AB000F8CF11C08091E8008B770BC08091AB02DA
:104AC000882349F08091E80080FFF8CF8091E800CA
:104AD0008E778093E80008952091E4003091E500FE
:104AE00095E64091EC00842F817040FF23C08091B7
:104AF000E80080FD1DC08091AB02882399F08530CD
:104B000099F08091EB0085FD11C04091E400509137
:104B1000E5002417350729F3915011F09A01E1CFF0
:104B200084E0089582E0089583E0089581E0089587
:104B300080E008954091E80042FFDDCF08950E9493
:104B40000D260E941526E0EEF0E0808181608083D2
:104B5000E8EDF0E080818F77808319BCA7EDB0E0AD
:104B60008C918E7F8C9380818F7E80831092AA029D
:104B700008950F931F93CF93DF930E940D260E94F9
:104B80001526C8EDD0E088818F778883888180687A
:104B9000888388818F7D888319BC1092AB02109224
:104BA000A7021092A9021092A80200EE10E0F801EC
:104BB00080818B7F808388818160888342E060E090
:104BC00080E00E941825E1EEF0E080818E7F8083F6
:104BD000E2EEF0E080818160808380818860808364
:104BE000F80180818E7F8083888180618883DF9156
:104BF000CF911F910F910895E8EDF0E080818F7EB5
:104C00008083E7EDF0E080818160808384E082BF73
:104C100081E08093AA020C94B925E8EDF0E0808150
:104C20008E7F80831092E20008951092DA00109235
:104C3000E10008951F920F920FB60F9211242F9347
:104C40003F934F935F936F937F938F939F93AF9314
:104C5000BF93EF93FF938091E10082FF0BC080919F
:104C6000E20082FF07C08091E1008B7F8093E1002A
:104C70000E94DD218091DA0080FF1FC08091D80062
:104C800080FF1BC08091DA008E7F8093DA008091D4
:104C9000D90080FF0DC080E189BD82E189BD09B4E2
:104CA00000FEFDCF81E08093AB020E94A42105C0ED
:104CB00019BC1092AB020E94B6218091E10080FFE6
:104CC00019C08091E20080FF15C08091E2008E7FC4
:104CD0008093E2008091E20080618093E200809105
:104CE000D80080628093D80019BC85E08093AB0225
:104CF0000E94C3218091E10084FF30C08091E200D6
:104D000084FF2CC080E189BD82E189BD09B400FE29
:104D1000FDCF8091D8008F7D8093D8008091E100F5
:104D20008F7E8093E1008091E2008F7E8093E2008D
:104D30008091E20081608093E2008091A702882345
:104D400011F084E007C08091E30087FD02C081E09C
:104D500001C083E08093AB020E94CF218091E100EB
:104D600083FF29C08091E20083FF25C08091E1008C
:104D7000877F8093E10082E08093AB021092A702CC
:104D80008091E1008E7F8093E1008091E2008E7F30
:104D90008093E2008091E20080618093E20042E033
:104DA00060E080E00E9418258091F0008860809388
:104DB000F0000E94BD21FF91EF91BF91AF919F91B3
:104DC0008F917F916F915F914F913F912F910F90B4
:104DD0000FBE0F901F9018951F920F920FB60F9253
:104DE00011242F933F934F935F936F937F938F93F0
:104DF0009F93AF93BF93CF93DF93EF93FF93C091B4
:104E0000E900CF708091EC00D82FD17080FDD0E800
:104E10001092E9008091F000877F8093F0007894F1
:104E20000E9430271092E9008091F0008860809302
:104E3000F000CD2BCF70C093E900FF91EF91DF918F
:104E4000CF91BF91AF919F918F917F916F915F9122
:104E50004F913F912F910F900FBE0F901F9018957B
:104E60001F93CF93DF93CDB7DEB7AA970FB6F89411
:104E7000DEBF0FBECDBFECEAF2E08091F10081937E
:104E800022E0E43BF207C9F70E9437228091E80054
:104E900083FF2EC18091AC029091AD02492F50E06A
:104EA0004A30510508F024C1FA01EE59FF4F0C9425
:104EB000CB28803821F0823809F01AC108C08091CF
:104EC000A8029091A902992389F082600FC0809175
:104ED000B0028F70873008F00BC18093E900809199
:104EE000EB0085FB882780F91092E9009091E8009B
:104EF000977F9093E8008093F1001092F100D1C069
:104F0000282F2D7F09F0F4C0882319F0823061F03A
:104F1000EFC08091AE02813009F0EAC0933009F011
:104F200080E08093A9022EC08091AE0281112AC038
:104F30008091B0028F702FEF280F263008F0D8C074
:104F40008093E9002091EB0020FF1CC0933021F4F6
:104F50008091EB00806214C09091EB00906190937F
:104F6000EB0021E030E0A90102C0440F551F8A95F3
:104F7000E2F74093EA001092EA008091EB0088602B
:104F80008093EB001092E9008091E800877F809386
:104F9000E8000E944D25ACC08111AAC01091AE025C
:104FA0001F778091E3008078812B8093E3008091CC
:104FB000E800877F8093E8000E944D258091E800FB
:104FC00080FFFCCF8091E30080688093E3001111A3
:104FD00002C082E001C083E08093AB0289C08058A8
:104FE000823008F085C08091AE029091AF028C3D76
:104FF00053E0950779F583E08A838AE289834FB786
:10500000F894DE01139620E03EE051E2E32FF0E059
:1050100050935700E49120FF03C0E295EF703F5F8B
:10502000EF708E2F90E0EA3010F0C79601C0C09666
:105030008D939D932F5F243149F74FBF8091E800F6
:10504000877F8093E8006AE270E0CE0101960E94BB
:10505000592416C06091B0027091B102AE014F5F49
:105060005F4F0E94A023BC01892B09F441C090919D
:10507000E800977F9093E80089819A810E94B72485
:105080008091E8008B778093E80032C0803881F50A
:105090008091E800877F8093E8008091A702809349
:1050A000F1008091E8008E7772CF811121C080914C
:1050B000AE029091AF0299270297D4F48091E80054
:1050C000877F8093E8008091AE028093A7020E94C0
:1050D0004D258091A702811106C08091E30087FDD4
:1050E00002C081E001C084E08093AB020E941E22D6
:1050F0008091E80083FF0AC08091E800877F809359
:10510000E8008091EB0080628093EB00AA960FB6D6
:10511000F894DEBF0FBECDBFDF91CF911F910895F0
:10512000CF938091AB028823A1F0C091E900CF70AA
:105130009091EC00892F817090FD80E8C82B10922F
:10514000E9008091E80083FD0E943027CF70C09372
:10515000E900CF910895991B79E004C0991F961733
:1051600008F0961B881F7A95C9F78095089597FBDC
:10517000072E16F4009407D077FD09D00E94D1289D
:1051800007FC05D03EF4909581959F4F089570954A
:1051900061957F4F0895EE0FFF1F0590F491E02D6C
:1051A0000994AA1BBB1B51E107C0AA1FBB1FA6176E
:1051B000B70710F0A61BB70B881F991F5A95A9F7C0
:1051C00080959095BC01CD010895FB01DC0104C0E0
:1051D0008D910190801921F441505040C8F7881BEF
:1051E000990B0895F999FECF92BD81BDF89A992740
:1051F00080B50895A8E1B0E042E050E00C94262983
:10520000262FF999FECF92BD81BDF89A019700B47F
:10521000021639F01FBA20BD0FB6F894FA9AF99A1F
:105220000FBE08950396272F0E9401290E9400298E
:10523000252F0E940129242F0C9401290196272F44
:105240000E9401290C940029DC01CB01FC01F99991
:10525000FECF06C0F2BDE1BDF89A319600B40D92C2
:0C52600041505040B8F70895F894FFCF7B
:10526C00C8004D02280850011E0A140122214521B4
:10527C002621A0219C21252101E200E900EA00B5AC
:10528C0000B600B700CD008301CC008A01920194D6
:10529C00012102230224022502260227022A02B33C
:1052AC0000B4006F007000818283E200E900EA0024
:1052BC00B500B600B700CD008301CC008A01920185
:1052CC0094012102230224022502260227022A022B
:1052DC00B300B4006F007000818283F6F73133663F
:1052EC0097C634353F3F3F006D6B5F64656C6179E9
:1052FC00006D6B5F696E74657276616C006D6B5FCF
:10530C006D61785F7370656564006D6B5F74696D5A
:10531C00655F746F5F6D6178006D6B5F7768656555
:10532C006C5F6D61785F7370656564006D6B5F7742
:10533C006865656C5F74696D655F746F5F6D6178CE
:10534C0000407B228B091009EE089308AC08C508B5
:00000001FF
